 gcstart002

 Timestamp is 3d9669ab (reproducible build file hash)

 Preferred load address is 0000000180000000

 Start         Length     Name                   Class
 0001:00000000 00003910H .text$mn                CODE
 0001:00003910 00000036H .text$mn$00             CODE
 0001:00003946 00000092H .text$x                 CODE
 0002:00000000 000001c8H .idata$5                DATA
 0002:000001c8 00000038H .00cfg                  DATA
 0002:00000200 00000008H .CRT$XCA                DATA
 0002:00000208 00000008H .CRT$XCZ                DATA
 0002:00000210 00000008H .CRT$XIA                DATA
 0002:00000218 00000008H .CRT$XIC                DATA
 0002:00000220 00000008H .CRT$XIZ                DATA
 0002:00000228 00000008H .CRT$XLA                DATA
 0002:00000230 00000008H .CRT$XLZ                DATA
 0002:00000238 00000008H .CRT$XPA                DATA
 0002:00000240 00000008H .CRT$XPZ                DATA
 0002:00000248 00000008H .CRT$XTA                DATA
 0002:00000250 00000010H .CRT$XTZ                DATA
 0002:00000258 00000000H .gehcont$y              DATA
 0002:00000258 00000000H .gfids$y                DATA
 0002:00000260 00002620H .rdata                  DATA
 0002:00002880 00000000H .rdata$CastGuardVftablesA DATA
 0002:00002880 00000000H .rdata$CastGuardVftablesC DATA
 0002:00002880 00000028H .rdata$T                DATA
 0002:000028a8 000000d0H .rdata$voltmd           DATA
 0002:00002978 00000318H .rdata$zzzdbg           DATA
 0002:00002c90 00000008H .rtc$IAA                DATA
 0002:00002c98 00000008H .rtc$IZZ                DATA
 0002:00002ca0 00000008H .rtc$TAA                DATA
 0002:00002ca8 00000008H .rtc$TZZ                DATA
 0002:00002cb0 00000004H .tls                    DATA
 0002:00002cb4 00000004H .tls$                   DATA
 0002:00002cb8 00000008H .tls$ZZZ                DATA
 0002:00002cc0 00000330H .xdata                  DATA
 0002:00002ff0 00000364H .edata                  DATA
 0002:00003354 0000008cH .idata$2                DATA
 0002:000033e0 00000018H .idata$3                DATA
 0002:000033f8 000001c8H .idata$4                DATA
 0002:000035c0 00000486H .idata$6                DATA
 0003:00000000 00000080H .data                   DATA
 0003:00000080 0001b398H .bss                    DATA
 0004:00000000 000003c0H .pdata                  DATA

  Address         Publics by Value              Rva+Base               Lib:Object

 0000:00000000       __AbsoluteZero             0000000000000000     <absolute>
 0000:00000000       ___safe_se_handler_count   0000000000000000     <absolute>
 0000:00000000       ___safe_se_handler_table   0000000000000000     <absolute>
 0000:00000000       __arm64x_extra_rfe_table   0000000000000000     <absolute>
 0000:00000000       __arm64x_extra_rfe_table_size 0000000000000000     <absolute>
 0000:00000000       __arm64x_native_entrypoint 0000000000000000     <absolute>
 0000:00000000       __arm64x_redirection_metadata 0000000000000000     <absolute>
 0000:00000000       __arm64x_redirection_metadata_count 0000000000000000     <absolute>
 0000:00000000       __dynamic_value_reloc_table 0000000000000000     <absolute>
 0000:00000000       __enclave_config           0000000000000000     <absolute>
 0000:00000000       __guard_check_icall_a64n_fptr 0000000000000000     <absolute>
 0000:00000000       __guard_eh_cont_count      0000000000000000     <absolute>
 0000:00000000       __guard_eh_cont_table      0000000000000000     <absolute>
 0000:00000000       __guard_fids_count         0000000000000000     <absolute>
 0000:00000000       __guard_fids_table         0000000000000000     <absolute>
 0000:00000000       __guard_iat_count          0000000000000000     <absolute>
 0000:00000000       __guard_iat_table          0000000000000000     <absolute>
 0000:00000000       __guard_longjmp_count      0000000000000000     <absolute>
 0000:00000000       __guard_longjmp_table      0000000000000000     <absolute>
 0000:00000000       __hybrid_auxiliary_iat     0000000000000000     <absolute>
 0000:00000000       __hybrid_auxiliary_iat_copy 0000000000000000     <absolute>
 0000:00000000       __hybrid_code_map          0000000000000000     <absolute>
 0000:00000000       __hybrid_code_map_count    0000000000000000     <absolute>
 0000:00000000       __x64_code_ranges_to_entry_points 0000000000000000     <absolute>
 0000:00000000       __x64_code_ranges_to_entry_points_count 0000000000000000     <absolute>
 0000:00000100       __guard_flags              0000000000000100     <absolute>
 0000:00000000       __ImageBase                0000000180000000     <linker-defined>
 0001:00000000       ?NewObject@JNIEnv_@@QEAAPEAV_jobject@@PEAV_jclass@@PEAU_jmethodID@@ZZ 0000000180001000 f i libgcstart002.obj
 0001:00000028       ?SetEventNotificationMode@_jvmtiEnv@@QEAA?AW4jvmtiError@@W4jvmtiEventMode@@W4jvmtiEvent@@PEAV_jobject@@ZZ 0000000180001028 f i libgcstart002.obj
 0001:00000034       ?TranslateError@@YAPEBDW4jvmtiError@@@Z 0000000180001034 f   libgcstart002.obj
 0001:000002ec       ?nsk_jni_check_exception@@YAHPEAUJNIEnv_@@QEBDH@Z 00000001800012ec f   libgcstart002.obj
 0001:00000430       ?nsk_jni_lverify@@YAHHPEAUJNIEnv_@@HQEBDH1ZZ 0000000180001430 f   libgcstart002.obj
 0001:000004d0       Agent_Initialize           00000001800014d0 f   libgcstart002.obj
 0001:00000848       Agent_OnAttach             0000000180001848 f   libgcstart002.obj
 0001:00000848       Agent_OnLoad               0000000180001848 f   libgcstart002.obj
 0001:00000850       GarbageCollectionStart     0000000180001850 f   libgcstart002.obj
 0001:00000a34       Java_nsk_jvmti_unit_FollowReferences_FollowRefObjects_addRefToVerify 0000000180001a34 f   libgcstart002.obj
 0001:00000c0c       Java_nsk_jvmti_unit_FollowReferences_FollowRefObjects_getTag 0000000180001c0c f   libgcstart002.obj
 0001:00000ccc       Java_nsk_jvmti_unit_FollowReferences_FollowRefObjects_resetRefsToVerify 0000000180001ccc f   libgcstart002.obj
 0001:00000cd4       Java_nsk_jvmti_unit_FollowReferences_FollowRefObjects_resetTags 0000000180001cd4 f   libgcstart002.obj
 0001:00000d18       Java_nsk_jvmti_unit_FollowReferences_FollowRefObjects_setTag 0000000180001d18 f   libgcstart002.obj
 0001:00000f70       Java_nsk_share_jvmti_ArgumentHandler_getAgentOptionsString 0000000180001f70 f   libgcstart002.obj
 0001:00001020       Java_nsk_share_jvmti_DebugeeClass_checkStatus 0000000180002020 f   libgcstart002.obj
 0001:000010a8       Java_nsk_share_jvmti_DebugeeClass_resetAgentData 00000001800020a8 f   libgcstart002.obj
 0001:00001108       Java_nsk_share_jvmti_RedefineAgent_agentStatus 0000000180002108 f   libgcstart002.obj
 0001:00001114       Java_nsk_share_jvmti_RedefineAgent_isRedefined 0000000180002114 f   libgcstart002.obj
 0001:00001120       Java_nsk_share_jvmti_RedefineAgent_redefineAttempted 0000000180002120 f   libgcstart002.obj
 0001:0000112c       MA_checkStatus             000000018000212c f   libgcstart002.obj
 0001:000011d0       VMDeath                    00000001800021d0 f   libgcstart002.obj
 0001:00001208       __local_stdio_printf_options 0000000180002208 f i libgcstart002.obj
 0001:000015ac       exitOnError                00000001800025ac f   libgcstart002.obj
 0001:00001660       fprintf                    0000000180002660 f i libgcstart002.obj
 0001:000016a4       nsk_complain               00000001800026a4 f   libgcstart002.obj
 0001:000016d0       nsk_jvmti_createJVMTIEnv   00000001800026d0 f   libgcstart002.obj
 0001:00001800       nsk_jvmti_lverify          0000000180002800 f   libgcstart002.obj
 0001:000018f0       nsk_jvmti_parseOptions     00000001800028f0 f   libgcstart002.obj
 0001:00001b40       nsk_jvmti_resetAgentData   0000000180002b40 f   libgcstart002.obj
 0001:00001bc0       nsk_jvmti_setFailStatus    0000000180002bc0 f   libgcstart002.obj
 0001:00001bfc       nsk_lcomplain              0000000180002bfc f   libgcstart002.obj
 0001:00001c1c       nsk_ldisplay               0000000180002c1c f   libgcstart002.obj
 0001:00001c3c       nsk_ltrace                 0000000180002c3c f   libgcstart002.obj
 0001:00001c5c       nsk_lvcomplain             0000000180002c5c f   libgcstart002.obj
 0001:00001e14       nsk_lvdisplay              0000000180002e14 f   libgcstart002.obj
 0001:00001e60       nsk_lverify                0000000180002e60 f   libgcstart002.obj
 0001:00001ebc       nsk_lvtrace                0000000180002ebc f   libgcstart002.obj
 0001:00001f1c       nsk_printf                 0000000180002f1c f   libgcstart002.obj
 0001:00001f44       nsk_vprintf                0000000180002f44 f   libgcstart002.obj
 0001:00001ff8       printf                     0000000180002ff8 f i libgcstart002.obj
 0001:000029e8       __raise_securityfailure    00000001800039e8 f   MSVCRT:gs_report.obj
 0001:00002a1c       __report_gsfailure         0000000180003a1c f   MSVCRT:gs_report.obj
 0001:00002c5c       __GSHandlerCheck           0000000180003c5c f   MSVCRT:gshandler.obj
 0001:00002c7c       __GSHandlerCheckCommon     0000000180003c7c f   MSVCRT:gshandler.obj
 0001:00002cf0       __security_check_cookie    0000000180003cf0 f   MSVCRT:amdsecgs.obj
 0001:00003030       _DllMainCRTStartup         0000000180004030 f   MSVCRT:dll_dllmain.obj
 0001:00003070       __scrt_acquire_startup_lock 0000000180004070 f   MSVCRT:utility.obj
 0001:000030ac       __scrt_dllmain_after_initialize_c 00000001800040ac f   MSVCRT:utility.obj
 0001:000030e0       __scrt_dllmain_before_initialize_c 00000001800040e0 f   MSVCRT:utility.obj
 0001:000030f8       __scrt_dllmain_crt_thread_attach 00000001800040f8 f   MSVCRT:utility.obj
 0001:00003120       __scrt_dllmain_crt_thread_detach 0000000180004120 f   MSVCRT:utility.obj
 0001:00003138       __scrt_dllmain_exception_filter 0000000180004138 f   MSVCRT:utility.obj
 0001:00003198       __scrt_dllmain_uninitialize_c 0000000180004198 f   MSVCRT:utility.obj
 0001:000031c8       __scrt_dllmain_uninitialize_critical 00000001800041c8 f   MSVCRT:utility.obj
 0001:000031dc       __scrt_initialize_crt      00000001800041dc f   MSVCRT:utility.obj
 0001:00003228       __scrt_initialize_onexit_tables 0000000180004228 f   MSVCRT:utility.obj
 0001:000032b4       __scrt_is_nonwritable_in_current_image 00000001800042b4 f   MSVCRT:utility.obj
 0001:0000334c       __scrt_release_startup_lock 000000018000434c f   MSVCRT:utility.obj
 0001:00003370       __scrt_uninitialize_crt    0000000180004370 f   MSVCRT:utility.obj
 0001:0000339c       _onexit                    000000018000439c f   MSVCRT:utility.obj
 0001:000033d8       atexit                     00000001800043d8 f   MSVCRT:utility.obj
 0001:000033f0       __crt_debugger_hook        00000001800043f0 f   MSVCRT:utility_desktop.obj
 0001:000033f8       __scrt_fastfail            00000001800043f8 f   MSVCRT:utility_desktop.obj
 0001:00003544       _guard_check_icall_nop     0000000180004544 f i MSVCRT:guard_support.obj
 0001:00003548       __security_init_cookie     0000000180004548 f   MSVCRT:gs_support.obj
 0001:000035f4       DllMain                    00000001800045f4 f   MSVCRT:dll_dllmain_stub.obj
 0001:00003618       ?__scrt_initialize_type_info@@YAXXZ 0000000180004618 f   MSVCRT:tncleanup.obj
 0001:00003628       ?__scrt_uninitialize_type_info@@YAXXZ 0000000180004628 f   MSVCRT:tncleanup.obj
 0001:00003634       __local_stdio_scanf_options 0000000180004634 f i MSVCRT:default_local_stdio_options.obj
 0001:0000363c       __scrt_initialize_default_local_stdio_options 000000018000463c f   MSVCRT:default_local_stdio_options.obj
 0001:00003658       __scrt_get_dyn_tls_init_callback 0000000180004658 f   MSVCRT:dyn_tls_init.obj
 0001:00003660       _RTC_Initialize            0000000180004660 f   MSVCRT:initsect.obj
 0001:0000369c       _RTC_Terminate             000000018000469c f   MSVCRT:initsect.obj
 0001:000036d8       __isa_available_init       00000001800046d8 f   MSVCRT:cpu_disp.obj
 0001:00003884       _get_startup_argv_mode     0000000180004884 f   MSVCRT:argv_mode.obj
 0001:0000388c       __scrt_is_ucrt_dll_in_use  000000018000488c f   MSVCRT:ucrt_detection.obj
 0001:000038a0       memcpy                     00000001800048a0 f   vcruntime:VCRUNTIME140.dll
 0001:000038a6       memset                     00000001800048a6 f   vcruntime:VCRUNTIME140.dll
 0001:000038ac       strchr                     00000001800048ac f   vcruntime:VCRUNTIME140.dll
 0001:000038b2       __C_specific_handler       00000001800048b2 f   vcruntime:VCRUNTIME140.dll
 0001:000038b8       __std_type_info_destroy_list 00000001800048b8 f   vcruntime:VCRUNTIME140.dll
 0001:000038be       strcmp                     00000001800048be f   ucrt:api-ms-win-crt-string-l1-1-0.dll
 0001:000038c4       strlen                     00000001800048c4 f   ucrt:api-ms-win-crt-string-l1-1-0.dll
 0001:000038ca       _initterm                  00000001800048ca f   ucrt:api-ms-win-crt-runtime-l1-1-0.dll
 0001:000038d0       _initterm_e                00000001800048d0 f   ucrt:api-ms-win-crt-runtime-l1-1-0.dll
 0001:000038d6       _seh_filter_dll            00000001800048d6 f   ucrt:api-ms-win-crt-runtime-l1-1-0.dll
 0001:000038dc       _configure_narrow_argv     00000001800048dc f   ucrt:api-ms-win-crt-runtime-l1-1-0.dll
 0001:000038e2       _initialize_narrow_environment 00000001800048e2 f   ucrt:api-ms-win-crt-runtime-l1-1-0.dll
 0001:000038e8       _initialize_onexit_table   00000001800048e8 f   ucrt:api-ms-win-crt-runtime-l1-1-0.dll
 0001:000038ee       _register_onexit_function  00000001800048ee f   ucrt:api-ms-win-crt-runtime-l1-1-0.dll
 0001:000038f4       _execute_onexit_table      00000001800048f4 f   ucrt:api-ms-win-crt-runtime-l1-1-0.dll
 0001:000038fa       _crt_atexit                00000001800048fa f   ucrt:api-ms-win-crt-runtime-l1-1-0.dll
 0001:00003900       _cexit                     0000000180004900 f   ucrt:api-ms-win-crt-runtime-l1-1-0.dll
 0001:00003908       __acrt_initialize          0000000180004908 f   MSVCRT:ucrt_stubs.obj
 0001:00003908       __acrt_thread_attach       0000000180004908 f   MSVCRT:ucrt_stubs.obj
 0001:00003908       __acrt_thread_detach       0000000180004908 f   MSVCRT:ucrt_stubs.obj
 0001:00003908       __acrt_uninitialize        0000000180004908 f   MSVCRT:ucrt_stubs.obj
 0001:00003908       __acrt_uninitialize_critical 0000000180004908 f   MSVCRT:ucrt_stubs.obj
 0001:00003908       __scrt_stub_for_acrt_initialize 0000000180004908 f   MSVCRT:ucrt_stubs.obj
 0001:00003908       __scrt_stub_for_acrt_thread_attach 0000000180004908 f   MSVCRT:ucrt_stubs.obj
 0001:00003908       __scrt_stub_for_acrt_thread_detach 0000000180004908 f   MSVCRT:ucrt_stubs.obj
 0001:00003908       __scrt_stub_for_acrt_uninitialize 0000000180004908 f   MSVCRT:ucrt_stubs.obj
 0001:00003908       __scrt_stub_for_acrt_uninitialize_critical 0000000180004908 f   MSVCRT:ucrt_stubs.obj
 0001:00003908       __vcrt_initialize          0000000180004908 f   MSVCRT:ucrt_stubs.obj
 0001:00003908       __vcrt_thread_attach       0000000180004908 f   MSVCRT:ucrt_stubs.obj
 0001:00003908       __vcrt_thread_detach       0000000180004908 f   MSVCRT:ucrt_stubs.obj
 0001:00003908       __vcrt_uninitialize        0000000180004908 f   MSVCRT:ucrt_stubs.obj
 0001:00003908       __vcrt_uninitialize_critical 0000000180004908 f   MSVCRT:ucrt_stubs.obj
 0001:0000390c       __scrt_stub_for_is_c_termination_complete 000000018000490c f   MSVCRT:ucrt_stubs.obj
 0001:0000390c       _is_c_termination_complete 000000018000490c f   MSVCRT:ucrt_stubs.obj
 0001:00003920       _guard_dispatch_icall_nop  0000000180004920 f   MSVCRT:guard_dispatch.obj
 0001:00003940       _guard_xfg_dispatch_icall_nop 0000000180004940 f   MSVCRT:guard_xfg_dispatch.obj
 0002:00000000       __imp_RtlCaptureContext    0000000180005000     kernel32:KERNEL32.dll
 0002:00000008       __imp_RtlLookupFunctionEntry 0000000180005008     kernel32:KERNEL32.dll
 0002:00000010       __imp_RtlVirtualUnwind     0000000180005010     kernel32:KERNEL32.dll
 0002:00000018       __imp_UnhandledExceptionFilter 0000000180005018     kernel32:KERNEL32.dll
 0002:00000020       __imp_SetUnhandledExceptionFilter 0000000180005020     kernel32:KERNEL32.dll
 0002:00000028       __imp_GetCurrentProcess    0000000180005028     kernel32:KERNEL32.dll
 0002:00000030       __imp_TerminateProcess     0000000180005030     kernel32:KERNEL32.dll
 0002:00000038       __imp_IsProcessorFeaturePresent 0000000180005038     kernel32:KERNEL32.dll
 0002:00000040       __imp_CloseHandle          0000000180005040     kernel32:KERNEL32.dll
 0002:00000048       __imp_InitializeCriticalSectionAndSpinCount 0000000180005048     kernel32:KERNEL32.dll
 0002:00000050       __imp_DeleteCriticalSection 0000000180005050     kernel32:KERNEL32.dll
 0002:00000058       __imp_CreateEventW         0000000180005058     kernel32:KERNEL32.dll
 0002:00000060       __imp_GetModuleHandleW     0000000180005060     kernel32:KERNEL32.dll
 0002:00000068       __imp_GetProcAddress       0000000180005068     kernel32:KERNEL32.dll
 0002:00000070       __imp_IsDebuggerPresent    0000000180005070     kernel32:KERNEL32.dll
 0002:00000078       __imp_QueryPerformanceCounter 0000000180005078     kernel32:KERNEL32.dll
 0002:00000080       __imp_GetCurrentProcessId  0000000180005080     kernel32:KERNEL32.dll
 0002:00000088       __imp_GetCurrentThreadId   0000000180005088     kernel32:KERNEL32.dll
 0002:00000090       __imp_GetSystemTimeAsFileTime 0000000180005090     kernel32:KERNEL32.dll
 0002:00000098       __imp_DisableThreadLibraryCalls 0000000180005098     kernel32:KERNEL32.dll
 0002:000000a0       __imp_InitializeSListHead  00000001800050a0     kernel32:KERNEL32.dll
 0002:000000a8       \177KERNEL32_NULL_THUNK_DATA 00000001800050a8     kernel32:KERNEL32.dll
 0002:000000b0       __imp_memcpy               00000001800050b0     vcruntime:VCRUNTIME140.dll
 0002:000000b8       __imp_memset               00000001800050b8     vcruntime:VCRUNTIME140.dll
 0002:000000c0       __imp_strchr               00000001800050c0     vcruntime:VCRUNTIME140.dll
 0002:000000c8       __imp___C_specific_handler 00000001800050c8     vcruntime:VCRUNTIME140.dll
 0002:000000d0       __imp___std_type_info_destroy_list 00000001800050d0     vcruntime:VCRUNTIME140.dll
 0002:000000d8       \177VCRUNTIME140_NULL_THUNK_DATA 00000001800050d8     vcruntime:VCRUNTIME140.dll
 0002:000000e0       __imp_strtol               00000001800050e0     ucrt:api-ms-win-crt-convert-l1-1-0.dll
 0002:000000e8       \177api-ms-win-crt-convert-l1-1-0_NULL_THUNK_DATA 00000001800050e8     ucrt:api-ms-win-crt-convert-l1-1-0.dll
 0002:000000f0       __imp_malloc               00000001800050f0     ucrt:api-ms-win-crt-heap-l1-1-0.dll
 0002:000000f8       __imp_free                 00000001800050f8     ucrt:api-ms-win-crt-heap-l1-1-0.dll
 0002:00000100       \177api-ms-win-crt-heap-l1-1-0_NULL_THUNK_DATA 0000000180005100     ucrt:api-ms-win-crt-heap-l1-1-0.dll
 0002:00000108       __imp__errno               0000000180005108     ucrt:api-ms-win-crt-runtime-l1-1-0.dll
 0002:00000110       __imp_exit                 0000000180005110     ucrt:api-ms-win-crt-runtime-l1-1-0.dll
 0002:00000118       __imp__cexit               0000000180005118     ucrt:api-ms-win-crt-runtime-l1-1-0.dll
 0002:00000120       __imp__crt_atexit          0000000180005120     ucrt:api-ms-win-crt-runtime-l1-1-0.dll
 0002:00000128       __imp__execute_onexit_table 0000000180005128     ucrt:api-ms-win-crt-runtime-l1-1-0.dll
 0002:00000130       __imp__register_onexit_function 0000000180005130     ucrt:api-ms-win-crt-runtime-l1-1-0.dll
 0002:00000138       __imp__initialize_onexit_table 0000000180005138     ucrt:api-ms-win-crt-runtime-l1-1-0.dll
 0002:00000140       __imp__initialize_narrow_environment 0000000180005140     ucrt:api-ms-win-crt-runtime-l1-1-0.dll
 0002:00000148       __imp__configure_narrow_argv 0000000180005148     ucrt:api-ms-win-crt-runtime-l1-1-0.dll
 0002:00000150       __imp__seh_filter_dll      0000000180005150     ucrt:api-ms-win-crt-runtime-l1-1-0.dll
 0002:00000158       __imp__initterm_e          0000000180005158     ucrt:api-ms-win-crt-runtime-l1-1-0.dll
 0002:00000160       __imp__initterm            0000000180005160     ucrt:api-ms-win-crt-runtime-l1-1-0.dll
 0002:00000168       \177api-ms-win-crt-runtime-l1-1-0_NULL_THUNK_DATA 0000000180005168     ucrt:api-ms-win-crt-runtime-l1-1-0.dll
 0002:00000170       __imp___acrt_iob_func      0000000180005170     ucrt:api-ms-win-crt-stdio-l1-1-0.dll
 0002:00000178       __imp_fflush               0000000180005178     ucrt:api-ms-win-crt-stdio-l1-1-0.dll
 0002:00000180       __imp___stdio_common_vsprintf 0000000180005180     ucrt:api-ms-win-crt-stdio-l1-1-0.dll
 0002:00000188       __imp___stdio_common_vfprintf 0000000180005188     ucrt:api-ms-win-crt-stdio-l1-1-0.dll
 0002:00000190       \177api-ms-win-crt-stdio-l1-1-0_NULL_THUNK_DATA 0000000180005190     ucrt:api-ms-win-crt-stdio-l1-1-0.dll
 0002:00000198       __imp_strcmp               0000000180005198     ucrt:api-ms-win-crt-string-l1-1-0.dll
 0002:000001a0       __imp__strdup              00000001800051a0     ucrt:api-ms-win-crt-string-l1-1-0.dll
 0002:000001a0       __imp_strdup               00000001800051a0     ucrt:api-ms-win-crt-string-l1-1-0.dll
 0002:000001a8       __imp_strlen               00000001800051a8     ucrt:api-ms-win-crt-string-l1-1-0.dll
 0002:000001b0       __imp_strpbrk              00000001800051b0     ucrt:api-ms-win-crt-string-l1-1-0.dll
 0002:000001b8       __imp_strncpy              00000001800051b8     ucrt:api-ms-win-crt-string-l1-1-0.dll
 0002:000001c0       \177api-ms-win-crt-string-l1-1-0_NULL_THUNK_DATA 00000001800051c0     ucrt:api-ms-win-crt-string-l1-1-0.dll
 0002:000001c8       __guard_check_icall_fptr   00000001800051c8     MSVCRT:guard_support.obj
 0002:000001d0       __guard_xfg_check_icall_fptr 00000001800051d0     MSVCRT:guard_support.obj
 0002:000001d8       __guard_dispatch_icall_fptr 00000001800051d8     MSVCRT:guard_support.obj
 0002:000001e0       __guard_xfg_dispatch_icall_fptr 00000001800051e0     MSVCRT:guard_support.obj
 0002:000001e8       __guard_xfg_table_dispatch_icall_fptr 00000001800051e8     MSVCRT:guard_support.obj
 0002:000001f0       __castguard_check_failure_os_handled_fptr 00000001800051f0     MSVCRT:guard_support.obj
 0002:000001f8       __guard_memcpy_fptr        00000001800051f8     vcruntime:softmemtag.obj
 0002:00000200       __xc_a                     0000000180005200     MSVCRT:initializers.obj
 0002:00000208       __xc_z                     0000000180005208     MSVCRT:initializers.obj
 0002:00000210       __xi_a                     0000000180005210     MSVCRT:initializers.obj
 0002:00000220       __xi_z                     0000000180005220     MSVCRT:initializers.obj
 0002:00000228       __xl_a                     0000000180005228     MSVCRT:tlssup.obj
 0002:00000230       __xl_z                     0000000180005230     MSVCRT:tlssup.obj
 0002:00000238       __xp_a                     0000000180005238     MSVCRT:initializers.obj
 0002:00000240       __xp_z                     0000000180005240     MSVCRT:initializers.obj
 0002:00000248       __xt_a                     0000000180005248     MSVCRT:initializers.obj
 0002:00000250       __xt_z                     0000000180005250     MSVCRT:initializers.obj
 0002:00000260       g_refKindStr               0000000180005260     libgcstart002.obj
 0002:00000410       ??_C@_09BPLDFGCI@unknown_0@ 0000000180005410     libgcstart002.obj
 0002:00000420       ??_C@_0BL@FPNMECJD@JVMTI_HEAP_REFERENCE_CLASS@ 0000000180005420     libgcstart002.obj
 0002:00000440       ??_C@_0BL@FKGKKLNM@JVMTI_HEAP_REFERENCE_FIELD@ 0000000180005440     libgcstart002.obj
 0002:00000460       ??_C@_0CD@CAEHCFJF@JVMTI_HEAP_REFERENCE_ARRAY_ELEM@ 0000000180005460     libgcstart002.obj
 0002:00000488       ??_C@_0CC@DNEBMCNK@JVMTI_HEAP_REFERENCE_CLASS_LOAD@ 0000000180005488     libgcstart002.obj
 0002:000004b0       ??_C@_0BN@CJMIPEBB@JVMTI_HEAP_REFERENCE_SIGNERS@ 00000001800054b0     libgcstart002.obj
 0002:000004d0       ??_C@_0CH@HBOIDPEB@JVMTI_HEAP_REFERENCE_PROTECTION@ 00000001800054d0     libgcstart002.obj
 0002:000004f8       ??_C@_0BP@MDKGDGKL@JVMTI_HEAP_REFERENCE_INTERFACE@ 00000001800054f8     libgcstart002.obj
 0002:00000518       ??_C@_0CC@JJMIHNJH@JVMTI_HEAP_REFERENCE_STATIC_FIE@ 0000000180005518     libgcstart002.obj
 0002:00000540       ??_C@_0CD@IDHEEGID@JVMTI_HEAP_REFERENCE_CONSTANT_P@ 0000000180005540     libgcstart002.obj
 0002:00000568       ??_C@_0CA@EFFCHNG@JVMTI_HEAP_REFERENCE_SUPERCLASS@ 0000000180005568     libgcstart002.obj
 0002:00000588       ??_C@_0L@PCDFHGCJ@unknown_11@ 0000000180005588     libgcstart002.obj
 0002:00000598       ??_C@_0L@NJBICFOK@unknown_12@ 0000000180005598     libgcstart002.obj
 0002:000005a8       ??_C@_0L@MAADBEKL@unknown_13@ 00000001800055a8     libgcstart002.obj
 0002:000005b8       ??_C@_0L@IPECICGM@unknown_14@ 00000001800055b8     libgcstart002.obj
 0002:000005c8       ??_C@_0L@JGFJLDCN@unknown_15@ 00000001800055c8     libgcstart002.obj
 0002:000005d8       ??_C@_0L@LNHEOAOO@unknown_16@ 00000001800055d8     libgcstart002.obj
 0002:000005e8       ??_C@_0L@KEGPNBKP@unknown_17@ 00000001800055e8     libgcstart002.obj
 0002:000005f8       ??_C@_0L@CDPHMNGA@unknown_18@ 00000001800055f8     libgcstart002.obj
 0002:00000608       ??_C@_0L@DKOMPMCB@unknown_19@ 0000000180005608     libgcstart002.obj
 0002:00000618       ??_C@_0L@OJGIPJDB@unknown_20@ 0000000180005618     libgcstart002.obj
 0002:00000628       ??_C@_0CA@KAOFNDEM@JVMTI_HEAP_REFERENCE_JNI_GLOBAL@ 0000000180005628     libgcstart002.obj
 0002:00000648       ??_C@_0CC@HPFAJBK@JVMTI_HEAP_REFERENCE_SYSTEM_CLA@ 0000000180005648     libgcstart002.obj
 0002:00000670       ??_C@_0BN@FDEGFOHC@JVMTI_HEAP_REFERENCE_MONITOR@ 0000000180005670     libgcstart002.obj
 0002:00000690       ??_C@_0CB@HKIBCMAJ@JVMTI_HEAP_REFERENCE_STACK_LOCA@ 0000000180005690     libgcstart002.obj
 0002:000006b8       ??_C@_0BP@EAACMMOE@JVMTI_HEAP_REFERENCE_JNI_LOCAL@ 00000001800056b8     libgcstart002.obj
 0002:000006d8       ??_C@_0BM@IJDEOGOE@JVMTI_HEAP_REFERENCE_THREAD@ 00000001800056d8     libgcstart002.obj
 0002:000006f8       ??_C@_0BL@EDGPPKC@JVMTI_HEAP_REFERENCE_OTHER@ 00000001800056f8     libgcstart002.obj
 0002:00000714       ??_C@_04BCJPDBDA@Code@     0000000180005714     libgcstart002.obj
 0002:00000720       ??_C@_0BA@OCLMCFKC@LineNumberTable@ 0000000180005720     libgcstart002.obj
 0002:00000730       ??_C@_0BD@CPAEPILC@LocalVariableTable@ 0000000180005730     libgcstart002.obj
 0002:00000748       ??_C@_0BH@NMBDNHBD@LocalVariableTypeTable@ 0000000180005748     libgcstart002.obj
 0002:00000760       ??_C@_0O@HIHEEDNJ@StackMapTable@ 0000000180005760     libgcstart002.obj
 0002:00000770       ??_C@_0L@HCDIAMJG@?9?5?$CFs?0?5?$CFd?3?5@ 0000000180005770     libgcstart002.obj
 0002:00000780       ??_C@_0JI@HLPECLFI@?$CD?5?4?4?4?6?$CD?5ERROR?3?5too?5many?5complai@ 0000000180005780     libgcstart002.obj
 0002:00000820       ??_C@_0ED@JNEKCCOB@The?5following?5fake?5exception?5st@ 0000000180005820     libgcstart002.obj
 0002:00000868       ??_C@_0CN@FCNMDFBH@nsk?4share?4Fake_Exception_for_RU@ 0000000180005868     libgcstart002.obj
 0002:00000898       ??_C@_08PGFFNAEI@?$CI?$CFs?3?$CFd?$CJ?5@ 0000000180005898     libgcstart002.obj
 0002:000008a8       ??_C@_0DP@IENMAEGI@s?2test?2hotspot?2jtreg?2vmTestbase@ 00000001800058a8     libgcstart002.obj
 0002:000008e8       ??_C@_0BL@NDJLFFJB@?7at?5nsk_lvcomplain?$CI?$CFs?3?$CFd?$CJ?6@ 00000001800058e8     libgcstart002.obj
 0002:00000908       ??_C@_0BC@JOOKAFKF@?$CD?5ERROR?3?5?$CFs?0?5?$CFd?3?5@ 0000000180005908     libgcstart002.obj
 0002:00000920       ??_C@_09KJEAHMEH@?$CD?5ERROR?3?5@ 0000000180005920     libgcstart002.obj
 0002:0000092c       ??_C@_02GPIOPFAK@?$DO?$DO@ 000000018000592c     libgcstart002.obj
 0002:00000930       ??_C@_02FODMEDOG@?$DM?$DM@ 0000000180005930     libgcstart002.obj
 0002:00000934       ??_C@_02DJGKEECL@?4?4@     0000000180005934     libgcstart002.obj
 0002:00000938       ??_C@_0O@CJPGJOAF@?9?5?$CFs?0?5?$CFd?3?5?$CFs?5@ 0000000180005938     libgcstart002.obj
 0002:00000948       ??_C@_0CB@IAKPDOIC@?$CD?5?5?5verified?5assertion?5is?5FALSE@ 0000000180005948     libgcstart002.obj
 0002:00000970       ??_C@_0CO@LGONDEPD@stdout?3?5fflush?5failed?5?9?5err?$DN?$CFd?5@ 0000000180005970     libgcstart002.obj
 0002:000009a0       ??_C@_0CO@KBGKJPBD@stderr?3?5fflush?5failed?5?9?5err?$DN?$CFd?5@ 00000001800059a0     libgcstart002.obj
 0002:000009d0       ??_C@_0BB@JCNMKLLK@JVMTI_ERROR_NONE@ 00000001800059d0     libgcstart002.obj
 0002:000009e8       ??_C@_0BL@LDIMKLPH@JVMTI_ERROR_INVALID_THREAD@ 00000001800059e8     libgcstart002.obj
 0002:00000a08       ??_C@_0CB@PJFPAIKJ@JVMTI_ERROR_INVALID_THREAD_GROU@ 0000000180005a08     libgcstart002.obj
 0002:00000a30       ??_C@_0BN@LLMKHMNF@JVMTI_ERROR_INVALID_PRIORITY@ 0000000180005a30     libgcstart002.obj
 0002:00000a50       ??_C@_0CB@MBOFKAGB@JVMTI_ERROR_THREAD_NOT_SUSPENDE@ 0000000180005a50     libgcstart002.obj
 0002:00000a78       ??_C@_0BN@FABOLPBI@JVMTI_ERROR_THREAD_SUSPENDED@ 0000000180005a78     libgcstart002.obj
 0002:00000a98       ??_C@_0BN@FDGNOBJM@JVMTI_ERROR_THREAD_NOT_ALIVE@ 0000000180005a98     libgcstart002.obj
 0002:00000ab8       ??_C@_0BL@GOBIFKNJ@JVMTI_ERROR_INVALID_OBJECT@ 0000000180005ab8     libgcstart002.obj
 0002:00000ad8       ??_C@_0BK@FCMAJPPC@JVMTI_ERROR_INVALID_CLASS@ 0000000180005ad8     libgcstart002.obj
 0002:00000af8       ??_C@_0BP@IKLLBKEB@JVMTI_ERROR_CLASS_NOT_PREPARED@ 0000000180005af8     libgcstart002.obj
 0002:00000b18       ??_C@_0BN@KLPPLKG@JVMTI_ERROR_INVALID_METHODID@ 0000000180005b18     libgcstart002.obj
 0002:00000b38       ??_C@_0BN@BCEKOKND@JVMTI_ERROR_INVALID_LOCATION@ 0000000180005b38     libgcstart002.obj
 0002:00000b58       ??_C@_0BM@DFDGPME@JVMTI_ERROR_INVALID_FIELDID@ 0000000180005b58     libgcstart002.obj
 0002:00000b78       ??_C@_0BL@NELIEPEC@JVMTI_ERROR_NO_MORE_FRAMES@ 0000000180005b78     libgcstart002.obj
 0002:00000b98       ??_C@_0BJ@BDBECFDM@JVMTI_ERROR_OPAQUE_FRAME@ 0000000180005b98     libgcstart002.obj
 0002:00000bb8       ??_C@_0BK@MIIFNLOB@JVMTI_ERROR_TYPE_MISMATCH@ 0000000180005bb8     libgcstart002.obj
 0002:00000bd8       ??_C@_0BJ@HPCAOILC@JVMTI_ERROR_INVALID_SLOT@ 0000000180005bd8     libgcstart002.obj
 0002:00000bf8       ??_C@_0BG@CHILOPNI@JVMTI_ERROR_DUPLICATE@ 0000000180005bf8     libgcstart002.obj
 0002:00000c10       ??_C@_0BG@DIEMLHKM@JVMTI_ERROR_NOT_FOUND@ 0000000180005c10     libgcstart002.obj
 0002:00000c28       ??_C@_0BM@NHMCKHOB@JVMTI_ERROR_INVALID_MONITOR@ 0000000180005c28     libgcstart002.obj
 0002:00000c48       ??_C@_0BO@PPEDAJGL@JVMTI_ERROR_NOT_MONITOR_OWNER@ 0000000180005c48     libgcstart002.obj
 0002:00000c68       ??_C@_0BG@FCAIPEID@JVMTI_ERROR_INTERRUPT@ 0000000180005c68     libgcstart002.obj
 0002:00000c80       ??_C@_0CB@EGDBNKOI@JVMTI_ERROR_INVALID_CLASS_FORMA@ 0000000180005c80     libgcstart002.obj
 0002:00000ca8       ??_C@_0CG@DGKOGIAL@JVMTI_ERROR_CIRCULAR_CLASS_DEFI@ 0000000180005ca8     libgcstart002.obj
 0002:00000cd0       ??_C@_0BP@ICEALPKC@JVMTI_ERROR_FAILS_VERIFICATION@ 0000000180005cd0     libgcstart002.obj
 0002:00000cf0       ??_C@_0DC@JDACLMIO@JVMTI_ERROR_UNSUPPORTED_REDEFIN@ 0000000180005cf0     libgcstart002.obj
 0002:00000d28       ??_C@_0DE@GKDKNOMJ@JVMTI_ERROR_UNSUPPORTED_REDEFIN@ 0000000180005d28     libgcstart002.obj
 0002:00000d60       ??_C@_0BO@LAFKIOG@JVMTI_ERROR_INVALID_TYPESTATE@ 0000000180005d60     libgcstart002.obj
 0002:00000d80       ??_C@_0DH@INDGCLLB@JVMTI_ERROR_UNSUPPORTED_REDEFIN@ 0000000180005d80     libgcstart002.obj
 0002:00000db8       ??_C@_0DE@NHEOMMGI@JVMTI_ERROR_UNSUPPORTED_REDEFIN@ 0000000180005db8     libgcstart002.obj
 0002:00000df0       ??_C@_0CA@EKPNJOEP@JVMTI_ERROR_UNSUPPORTED_VERSION@ 0000000180005df0     libgcstart002.obj
 0002:00000e10       ??_C@_0BN@OFFMAHHL@JVMTI_ERROR_NAMES_DONT_MATCH@ 0000000180005e10     libgcstart002.obj
 0002:00000e30       ??_C@_0DN@HHBBLAKE@JVMTI_ERROR_UNSUPPORTED_REDEFIN@ 0000000180005e30     libgcstart002.obj
 0002:00000e70       ??_C@_0DO@HMBGBGNA@JVMTI_ERROR_UNSUPPORTED_REDEFIN@ 0000000180005e70     libgcstart002.obj
 0002:00000eb0       ??_C@_0BP@PBECGKHJ@JVMTI_ERROR_UNMODIFIABLE_CLASS@ 0000000180005eb0     libgcstart002.obj
 0002:00000ed0       ??_C@_0BK@CANILEHF@JVMTI_ERROR_NOT_AVAILABLE@ 0000000180005ed0     libgcstart002.obj
 0002:00000ef0       ??_C@_0CE@INJKMEFK@JVMTI_ERROR_MUST_POSSESS_CAPABI@ 0000000180005ef0     libgcstart002.obj
 0002:00000f18       ??_C@_0BJ@LBFPFPDM@JVMTI_ERROR_NULL_POINTER@ 0000000180005f18     libgcstart002.obj
 0002:00000f38       ??_C@_0BP@CHJPNNEM@JVMTI_ERROR_ABSENT_INFORMATION@ 0000000180005f38     libgcstart002.obj
 0002:00000f58       ??_C@_0BP@OMFMNLC@JVMTI_ERROR_INVALID_EVENT_TYPE@ 0000000180005f58     libgcstart002.obj
 0002:00000f78       ??_C@_0BN@BIBNPHHO@JVMTI_ERROR_ILLEGAL_ARGUMENT@ 0000000180005f78     libgcstart002.obj
 0002:00000f98       ??_C@_0BK@KKNDHDCE@JVMTI_ERROR_NATIVE_METHOD@ 0000000180005f98     libgcstart002.obj
 0002:00000fb8       ??_C@_0BK@PMKCFHAE@JVMTI_ERROR_OUT_OF_MEMORY@ 0000000180005fb8     libgcstart002.obj
 0002:00000fd8       ??_C@_0BK@NNJBDMNB@JVMTI_ERROR_ACCESS_DENIED@ 0000000180005fd8     libgcstart002.obj
 0002:00000ff8       ??_C@_0BI@GHECLMNC@JVMTI_ERROR_WRONG_PHASE@ 0000000180005ff8     libgcstart002.obj
 0002:00001010       ??_C@_0BF@OLIHJOII@JVMTI_ERROR_INTERNAL@ 0000000180006010     libgcstart002.obj
 0002:00001028       ??_C@_0BO@EOHGKJHI@JVMTI_ERROR_UNATTACHED_THREAD@ 0000000180006028     libgcstart002.obj
 0002:00001048       ??_C@_0CA@LKHFDACL@JVMTI_ERROR_INVALID_ENVIRONMENT@ 0000000180006048     libgcstart002.obj
 0002:00001068       ??_C@_0BA@MMFHLOKK@?$DMunknown?5error?$DO@ 0000000180006068     libgcstart002.obj
 0002:00001078       ??_C@_0CF@CBHOKDB@throwable?5?$DN?5jni?9?$DOExceptionOccur@ 0000000180006078     libgcstart002.obj
 0002:000010a0       ??_C@_03OFAPEBGM@?$CFs?6@  00000001800060a0     libgcstart002.obj
 0002:000010a8       ??_C@_0DM@LPIGEGNJ@s?2test?2hotspot?2jtreg?2vmTestbase@ 00000001800060a8     libgcstart002.obj
 0002:000010e8       ??_C@_0CC@NFCNPEPK@Exception?5in?5JNI?5call?5?$CIcleared?$CJ@ 00000001800060e8     libgcstart002.obj
 0002:00001110       ??_C@_0BJ@IBAKFIKF@jni?9?$DOExceptionDescribe?$CI?$CJ@ 0000000180006110     libgcstart002.obj
 0002:00001130       ??_C@_0BG@GGKALKMH@jni?9?$DOExceptionClear?$CI?$CJ@ 0000000180006130     libgcstart002.obj
 0002:00001148       ??_C@_0CF@JMGFGJLJ@?$CD?5?5?5verified?5JNI?5assertion?5is?5F@ 0000000180006148     libgcstart002.obj
 0002:00001170       ??_C@_07KBAMPNJK@verbose@  0000000180006170     libgcstart002.obj
 0002:00001178       ??_C@_0DN@PKJBOLAP@nsk_jvmti_parseOptions?$CI?$CJ?3?5unexp@ 0000000180006178     libgcstart002.obj
 0002:000011b8       ??_C@_05IMBNNINJ@trace@    00000001800061b8     libgcstart002.obj
 0002:000011c0       ??_C@_0DD@BJKGNDMB@nsk_jvmti_parseOptions?$CI?$CJ?3?5no?5va@ 00000001800061c0     libgcstart002.obj
 0002:000011f4       ??_C@_04CGFJFPFD@none@     00000001800061f4     libgcstart002.obj
 0002:000011fc       ??_C@_06BMELKFMA@before@   00000001800061fc     libgcstart002.obj
 0002:00001204       ??_C@_05CMKPCFDK@after@    0000000180006204     libgcstart002.obj
 0002:0000120c       ??_C@_03NFKEKGGK@all@      000000018000620c     libgcstart002.obj
 0002:00001210       ??_C@_0DM@NDNJGJKE@nsk_jvmti_parseOptions?$CI?$CJ?3?5uexpe@ 0000000180006210     libgcstart002.obj
 0002:00001250       ??_C@_08NBBJKJO@waittime@  0000000180006250     libgcstart002.obj
 0002:00001260       ??_C@_0DO@CMHGAOHC@nsk_jvmti_parseOptions?$CI?$CJ?3?5not?5i@ 0000000180006260     libgcstart002.obj
 0002:000012a0       ??_C@_0DL@LNMPBDLN@nsk_jvmti_parseOptions?$CI?$CJ?3?5negat@ 00000001800062a0     libgcstart002.obj
 0002:000012e0       ??_C@_0DA@GMFJNOJH@nsk_jvmti_parseOptions?$CI?$CJ?3?5unkno@ 00000001800062e0     libgcstart002.obj
 0002:00001310       ??_C@_0CO@CCIAMEAN@nsk_jvmti_parseOptions?$CI?$CJ?3?5found@ 0000000180006310     libgcstart002.obj
 0002:00001340       ??_C@_0CJ@OEGPCGDL@nsk_jvmti_parseOptions?$CI?$CJ?3?5out?5o@ 0000000180006340     libgcstart002.obj
 0002:00001370       ??_C@_0DI@NMBHPGGF@nsk_jvmti_parseOptions?$CI?$CJ?3?5too?5m@ 0000000180006370     libgcstart002.obj
 0002:000013a8       ??_C@_03POGCGECB@?5?0?$HO@ 00000001800063a8     libgcstart002.obj
 0002:000013b0       ??_C@_0CB@MLNJNCLJ@?5?5jvmti?5error?3?5code?$DN?$CFd?0?5name?$DN?$CFs@ 00000001800063b0     libgcstart002.obj
 0002:000013d8       ??_C@_0CD@OHBGDKMK@?$CD?5?5?5jvmti?5error?3?5code?$DN?$CFd?0?5name?$DN@ 00000001800063d8     libgcstart002.obj
 0002:00001400       ??_C@_0CG@JNNCGPHB@?$CD?5?5?5error?5expected?3?5code?$DN?$CFd?0?5na@ 0000000180006400     libgcstart002.obj
 0002:00001430       ??_C@_0EB@IMGKPCGE@?$CIstr_obj?5?$DN?5jni?9?$DONewStringUTF?$CIco@ 0000000180006430     libgcstart002.obj
 0002:00001480       ??_C@_0EA@HFOGGBCC@s?2test?2hotspot?2jtreg?2vmTestbase@ 0000000180006480     libgcstart002.obj
 0002:000014c0       ??_C@_05KKCIMGE@error@     00000001800064c0     libgcstart002.obj
 0002:000014c8       ??_C@_0CJ@JACLEAA@Test?5failed?5by?5setFailStatus?$CI?$CJ?4@ 00000001800064c8     libgcstart002.obj
 0002:000014f8       ??_C@_0BD@HGNAOMCP@agent_data_monitor@ 00000001800064f8     libgcstart002.obj
 0002:00001510       ??_C@_0EB@OGCLGKLN@javaVM?9?$DOGetEnv?$CI?$CIvoid?5?$CK?$CK?$CJ?$CGjvmti_@ 0000000180006510     libgcstart002.obj
 0002:00001560       ??_C@_0EA@PNBCDMOA@s?2test?2hotspot?2jtreg?2vmTestbase@ 0000000180006560     libgcstart002.obj
 0002:000015a0       ??_C@_0CI@DDPIFBGM@init_agent_data?$CIjvmti_env?0?5?$CGage@ 00000001800065a0     libgcstart002.obj
 0002:000015c8       ??_C@_0DI@ILAHDLMP@?$CI?$CKagentThreadProc?$CJ?$CIjvmti_env?0?5a@ 00000001800065c8     libgcstart002.obj
 0002:00001600       ??_C@_0BD@KDBALNLB@JVMTI?5agent?5thread@ 0000000180006600     libgcstart002.obj
 0002:00001618       ??_C@_0BB@NOKBFPFO@java?1lang?1Thread@ 0000000180006618     libgcstart002.obj
 0002:0000162c       ??_C@_06FALKBLGB@?$DMinit?$DO@ 000000018000662c     libgcstart002.obj
 0002:00001638       ??_C@_0BG@IKDDPPGD@?$CILjava?1lang?1String?$DL?$CJV@ 0000000180006638     libgcstart002.obj
 0002:00001650       ??_C@_0EB@IFJBFEKC@?$CIthreadClass?5?$DN?5jni_env?9?$DOFindCla@ 0000000180006650     libgcstart002.obj
 0002:000016a0       ??_C@_0GF@FGFIBKKL@?$CIthreadCtor?5?$DN?5jni_env?9?$DOGetMetho@ 00000001800066a0     libgcstart002.obj
 0002:00001708       ??_C@_0DN@NCPDJLOG@?$CIthreadName?5?$DN?5jni_env?9?$DONewStrin@ 0000000180006708     libgcstart002.obj
 0002:00001750       ??_C@_0FE@PFKODBGC@?$CIthreadObject?5?$DN?5jni_env?9?$DONewObj@ 0000000180006750     libgcstart002.obj
 0002:000017b0       ??_C@_0ED@HOBAHHJI@?$CIthreadGlobalRef?5?$DN?5jni_env?9?$DONew@ 00000001800067b0     libgcstart002.obj
 0002:00001800       ??_C@_0FN@HNJJAHFC@jvmti_env?9?$DORunAgentThread?$CIagent@ 0000000180006800     libgcstart002.obj
 0002:00001860       ??_C@_0EA@MOJDNKDF@Debuggee?5status?5sync?5aborted?5be@ 0000000180006860     libgcstart002.obj
 0002:000018a0       ??_C@_0EA@EEOEJAEN@status?5?$DN?5syncDebuggeeStatus?$CIjni@ 00000001800068a0     libgcstart002.obj
 0002:000018e0       ??_C@_0BL@JBCFNBMB@nsk_jvmti_resetAgentData?$CI?$CJ@ 00000001800068e0     libgcstart002.obj
 0002:00001900       ??_C@_0EL@LPBEELIP@s?2test?2hotspot?2jtreg?2vmTestbase@ 0000000180006900     libgcstart002.obj
 0002:00001950       ??_C@_0CK@JDAMFDMJ@jvmti?9?$DOSetTag?$CIo?0?5tag?$CJ?5?$DN?$DN?5JVMTI_@ 0000000180006950     libgcstart002.obj
 0002:00001980       ??_C@_0CC@DAMNHKNI@Can?8t?5set?5tag?5?$CFli?5for?5object?5?$CFl@ 0000000180006980     libgcstart002.obj
 0002:000019a8       ??_C@_0DL@HAJPNKEF@jvmti?9?$DOGetObjectHashCode?$CIo?0?5?$CGha@ 00000001800069a8     libgcstart002.obj
 0002:000019e8       ??_C@_0BL@JFPIEOBF@Can?8t?5get?5hash?5object?5?$CFlx?6@ 00000001800069e8     libgcstart002.obj
 0002:00001a08       ??_C@_0BG@DICPHBKN@setTag?3?5?$CF08x?5?$DM?9?5?$CF?53li@ 0000000180006a08     libgcstart002.obj
 0002:00001a20       ??_C@_0DH@FCEEBDMJ@?$CIs?5?$DN?5jni?9?$DOGetStringUTFChars?$CIsIn@ 0000000180006a20     libgcstart002.obj
 0002:00001a58       ??_C@_0BJ@OKKGHDCN@Can?8t?5get?5string?5at?5?$CF?$CDp?6@ 0000000180006a58     libgcstart002.obj
 0002:00001a78       ??_C@_0BP@EKFLGGFJ@Can?8t?5get?5string?5at?5?$CF?$CDp?3?5null?6@ 0000000180006a78     libgcstart002.obj
 0002:00001a98       ??_C@_06ICODBHCL@?5?1?1?5?$CFs@ 0000000180006a98     libgcstart002.obj
 0002:00001aa0       ??_C@_0DB@KGFPLEGO@?$CIr?5?$DN?5jvmti?9?$DOGetTag?$CIo?0?5?$CGtag?$CJ?$CJ?5?$DN?$DN@ 0000000180006aa0     libgcstart002.obj
 0002:00001ad8       ??_C@_0CO@PDAGBCGJ@Can?8t?5GetTag?5for?5object?5?$CFlx?4?5Re@ 0000000180006ad8     libgcstart002.obj
 0002:00001b08       ??_C@_0CH@HPEODOHC@TEST_BUG?3?5Max?4?5number?5of?5refs?5r@ 0000000180006b08     libgcstart002.obj
 0002:00001b30       ??_C@_0DI@PHFCABIM@?$CIr?5?$DN?5jvmti?9?$DOGetTag?$CIfrom?0?5?$CGtagFr@ 0000000180006b30     libgcstart002.obj
 0002:00001b68       ??_C@_0DI@MDEGFNKD@TEST_BUG?3?5Can?8t?5GetTag?5for?5obje@ 0000000180006b68     libgcstart002.obj
 0002:00001ba0       ??_C@_0DE@MLELJAHM@?$CIr?5?$DN?5jvmti?9?$DOGetTag?$CIto?0?5?$CGtagTo?$CJ?$CJ@ 0000000180006ba0     libgcstart002.obj
 0002:00001bd8       ??_C@_0CA@NFFMLHN@?$CFs?3?5creating?5a?5raw?5monitor?5?4?4?4?6@ 0000000180006bd8     libgcstart002.obj
 0002:00001c00       ??_C@_0FL@HAIPAEND@s?2test?2hotspot?2jtreg?2vmTestbase@ 0000000180006c00     libgcstart002.obj
 0002:00001c60       ??_C@_0CN@GMOGLIIN@jvmti_env?9?$DOCreateRawMonitor?$CI?$CC_l@ 0000000180006c60     libgcstart002.obj
 0002:00001c90       ??_C@_05EAPKFOHC@_lock@    0000000180006c90     libgcstart002.obj
 0002:00001c98       ??_C@_0DC@BFAML@TEST?5FAILED?3?5?$CFs?3?5unable?5to?5crea@ 0000000180006c98     libgcstart002.obj
 0002:00001cd0       ??_C@_0CH@ELPNCNMM@CHECK?5PASSED?3?5?$CFs?3?5raw?5monitor?5c@ 0000000180006cd0     libgcstart002.obj
 0002:00001cf8       ??_C@_0CC@KPNBIBOK@?$CFs?3?5entering?5the?5raw?5monitor?5?4?4@ 0000000180006cf8     libgcstart002.obj
 0002:00001d20       ??_C@_0CC@LICKJMEG@jvmti_env?9?$DORawMonitorEnter?$CI_loc@ 0000000180006d20     libgcstart002.obj
 0002:00001d48       ??_C@_0DD@ILNKINHA@TEST?5FAILED?3?5?$CFs?3?5unable?5to?5ente@ 0000000180006d48     libgcstart002.obj
 0002:00001d80       ??_C@_0CL@HOBMHNLB@CHECK?5PASSED?3?5?$CFs?3?5the?5raw?5monit@ 0000000180006d80     libgcstart002.obj
 0002:00001db0       ??_C@_0CB@CKCFLCHC@?$CFs?3?5waiting?5the?5raw?5monitor?5?4?4?4@ 0000000180006db0     libgcstart002.obj
 0002:00001dd8       ??_C@_0CM@JCJEGOIK@jvmti_env?9?$DORawMonitorWait?$CI_lock@ 0000000180006dd8     libgcstart002.obj
 0002:00001e08       ??_C@_0DC@HEFDLADG@TEST?5FAILED?3?5?$CFs?3?5unable?5to?5wait@ 0000000180006e08     libgcstart002.obj
 0002:00001e40       ??_C@_0CK@FALIEPOD@CHECK?5PASSED?3?5?$CFs?3?5the?5raw?5monit@ 0000000180006e40     libgcstart002.obj
 0002:00001e70       ??_C@_0DO@LEDIEDGM@?$CFs?3?5notifying?5a?5single?5thread?5w@ 0000000180006e70     libgcstart002.obj
 0002:00001eb0       ??_C@_0CD@MCEJJMHC@jvmti_env?9?$DORawMonitorNotify?$CI_lo@ 0000000180006eb0     libgcstart002.obj
 0002:00001ed8       ??_C@_0DC@NDHFJDDN@TEST?5FAILED?3?5?$CFs?3?5unable?5to?5noti@ 0000000180006ed8     libgcstart002.obj
 0002:00001f10       ??_C@_0CK@MNPOBPIB@CHECK?5PASSED?3?5?$CFs?3?5single?5thread@ 0000000180006f10     libgcstart002.obj
 0002:00001f40       ??_C@_0DK@BAPFBNKN@?$CFs?3?5notifying?5all?5threads?5waiti@ 0000000180006f40     libgcstart002.obj
 0002:00001f80       ??_C@_0CG@ICKGGLBM@jvmti_env?9?$DORawMonitorNotifyAll?$CI@ 0000000180006f80     libgcstart002.obj
 0002:00001fa8       ??_C@_0DA@KDBFDPJM@TEST?5FAILED?3?5?$CFs?3?5unable?5to?5noti@ 0000000180006fa8     libgcstart002.obj
 0002:00001fd8       ??_C@_0CI@LELHIBGI@CHECK?5PASSED?3?5?$CFs?3?5all?5threads?5n@ 0000000180006fd8     libgcstart002.obj
 0002:00002000       ??_C@_0CB@HNKHEJBK@?$CFs?3?5exiting?5the?5raw?5monitor?5?4?4?4@ 0000000180007000     libgcstart002.obj
 0002:00002028       ??_C@_0CB@FEMOEOEG@jvmti_env?9?$DORawMonitorExit?$CI_lock@ 0000000180007028     libgcstart002.obj
 0002:00002050       ??_C@_0DC@JPCLONBC@TEST?5FAILED?3?5?$CFs?3?5unable?5to?5exit@ 0000000180007050     libgcstart002.obj
 0002:00002088       ??_C@_0CK@JMGAKAKI@CHECK?5PASSED?3?5?$CFs?3?5the?5raw?5monit@ 0000000180007088     libgcstart002.obj
 0002:000020b8       ??_C@_0CE@KLCCECNE@?$CFs?3?5destroying?5the?5raw?5monitor?5@ 00000001800070b8     libgcstart002.obj
 0002:000020e0       ??_C@_0CE@LMOOLBIH@jvmti_env?9?$DODestroyRawMonitor?$CI_l@ 00000001800070e0     libgcstart002.obj
 0002:00002108       ??_C@_0DC@PKLDHPCH@TEST?5FAILED?3?5?$CFs?3?5unable?5to?5dest@ 0000000180007108     libgcstart002.obj
 0002:00002140       ??_C@_0CN@NBOLIIFJ@CHECK?5PASSED?3?5?$CFs?3?5the?5raw?5monit@ 0000000180007140     libgcstart002.obj
 0002:00002170       ??_C@_0BL@EDKNLHDL@?$CFs?3?5allocating?5memory?5?4?4?4?6@ 0000000180007170     libgcstart002.obj
 0002:00002190       ??_C@_0CE@DFLKJLND@jvmti_env?9?$DOAllocate?$CIMEM_SIZE?0?5?$CG@ 0000000180007190     libgcstart002.obj
 0002:000021b8       ??_C@_0CN@BDGANOPB@TEST?5FAILED?3?5?$CFs?3?5unable?5to?5allo@ 00000001800071b8     libgcstart002.obj
 0002:000021e8       ??_C@_0DK@KLGPKMFP@CHECK?5PASSED?3?5?$CFs?3?5memory?5has?5be@ 00000001800071e8     libgcstart002.obj
 0002:00002228       ??_C@_0BN@EKKCBNLG@?$CFs?3?5deallocating?5memory?5?4?4?4?6@ 0000000180007228     libgcstart002.obj
 0002:00002248       ??_C@_0BL@KHDPKCEF@jvmti_env?9?$DODeallocate?$CImem?$CJ@ 0000000180007248     libgcstart002.obj
 0002:00002268       ??_C@_0CP@PGMPPCAM@TEST?5FAILED?3?5?$CFs?3?5unable?5to?5deal@ 0000000180007268     libgcstart002.obj
 0002:00002298       ??_C@_0DN@HDLOEOCD@CHECK?5PASSED?3?5?$CFs?3?5memory?5has?5be@ 0000000180007298     libgcstart002.obj
 0002:000022d8       ??_C@_0DA@MMHBNCBI@?$DO?$DO?$DO?$DO?5GarbageCollectionStart?5eve@ 00000001800072d8     libgcstart002.obj
 0002:00002308       ??_C@_0BH@CBKEHIKC@GarbageCollectionStart@ 0000000180007308     libgcstart002.obj
 0002:00002320       ??_C@_06FHLMFHLD@?$DM?$DM?$DM?$DM?6?6@ 0000000180007320     libgcstart002.obj
 0002:00002328       ??_C@_0BI@OPPGFBGD@VMDeath?5event?5received?6@ 0000000180007328     libgcstart002.obj
 0002:00002340       ??_C@_0CA@MNKGCBCG@nsk_jvmti_parseOptions?$CIoptions?$CJ@ 0000000180007340     libgcstart002.obj
 0002:00002360       ??_C@_0DN@MIAMNFPH@?$CIjvmti?5?$DN?5nsk_jvmti_createJVMTIE@ 0000000180007360     libgcstart002.obj
 0002:000023a0       ??_C@_0BO@DBKDIPGD@jvmti?9?$DOAddCapabilities?$CI?$CGcaps?$CJ@ 00000001800073a0     libgcstart002.obj
 0002:000023c0       ??_C@_0BO@IAKFILDF@jvmti?9?$DOGetCapabilities?$CI?$CGcaps?$CJ@ 00000001800073c0     libgcstart002.obj
 0002:000023e0       ??_C@_0EF@PAKPNIJC@Warning?3?5generation?5of?5garbage?5@ 00000001800073e0     libgcstart002.obj
 0002:00002428       ??_C@_0BN@HGIKGGD@setting?5event?5callbacks?5?4?4?4?6@ 0000000180007428     libgcstart002.obj
 0002:00002448       ??_C@_0DI@NJCFGEGC@jvmti?9?$DOSetEventCallbacks?$CI?$CGcallb@ 0000000180007448     libgcstart002.obj
 0002:00002480       ??_C@_0DI@LEFDPPF@setting?5event?5callbacks?5done?6en@ 0000000180007480     libgcstart002.obj
 0002:000024c0       ??_C@_0EN@OLHGIFGG@jvmti?9?$DOSetEventNotificationMode@ 00000001800074c0     libgcstart002.obj
 0002:00002510       ??_C@_0FN@HGACOBCB@jvmti?9?$DOSetEventNotificationMode@ 0000000180007510     libgcstart002.obj
 0002:00002570       ??_C@_0BL@GBOGNFCP@enabling?5the?5events?5done?6?6@ 0000000180007570     libgcstart002.obj
 0002:000025a0       ??_C@_1EC@JIJBPKFM@?$AAa?$AAp?$AAi?$AA?9?$AAm?$AAs?$AA?9?$AAw?$AAi?$AAn?$AA?9?$AAc?$AAo?$AAr?$AAe@ 00000001800075a0     MSVCRT:thread_safe_statics.obj
 0002:000025e8       ??_C@_1BK@MGMFAEKH@?$AAk?$AAe?$AAr?$AAn?$AAe?$AAl?$AA3?$AA2?$AA?4?$AAd?$AAl?$AAl@ 00000001800075e8     MSVCRT:thread_safe_statics.obj
 0002:00002608       ??_C@_0BJ@JEBJOJFJ@SleepConditionVariableCS@ 0000000180007608     MSVCRT:thread_safe_statics.obj
 0002:00002628       ??_C@_0BJ@PGPPEPCC@WakeAllConditionVariable@ 0000000180007628     MSVCRT:thread_safe_statics.obj
 0002:00002648       _pDefaultRawDllMain        0000000180007648     MSVCRT:dll_dllmain.obj
 0002:00002648       _pRawDllMain               0000000180007648     MSVCRT:dll_dllmain.obj
 0002:00002650       __xmm@ffffffffffffffffffffffffffffffff 0000000180007650     MSVCRT:utility.obj
 0002:00002660       _load_config_used          0000000180007660     MSVCRT:loadcfg.obj
 0002:00002880       _tls_used                  0000000180007880     MSVCRT:tlssup.obj
 0002:000028a8       __volatile_metadata        00000001800078a8     <linker-defined>
 0002:00002c90       __rtc_iaa                  0000000180007c90     MSVCRT:initsect.obj
 0002:00002c98       __rtc_izz                  0000000180007c98     MSVCRT:initsect.obj
 0002:00002ca0       __rtc_taa                  0000000180007ca0     MSVCRT:initsect.obj
 0002:00002ca8       __rtc_tzz                  0000000180007ca8     MSVCRT:initsect.obj
 0002:00002cb0       _tls_start                 0000000180007cb0     MSVCRT:tlssup.obj
 0002:00002cb4       _Init_thread_epoch         0000000180007cb4     MSVCRT:thread_safe_statics.obj
 0002:00002cb8       _tls_end                   0000000180007cb8     MSVCRT:tlssup.obj
 0002:00003354       __IMPORT_DESCRIPTOR_KERNEL32 0000000180008354     kernel32:KERNEL32.dll
 0002:00003368       __IMPORT_DESCRIPTOR_VCRUNTIME140 0000000180008368     vcruntime:VCRUNTIME140.dll
 0002:0000337c       __IMPORT_DESCRIPTOR_api-ms-win-crt-heap-l1-1-0 000000018000837c     ucrt:api-ms-win-crt-heap-l1-1-0.dll
 0002:00003390       __IMPORT_DESCRIPTOR_api-ms-win-crt-runtime-l1-1-0 0000000180008390     ucrt:api-ms-win-crt-runtime-l1-1-0.dll
 0002:000033a4       __IMPORT_DESCRIPTOR_api-ms-win-crt-convert-l1-1-0 00000001800083a4     ucrt:api-ms-win-crt-convert-l1-1-0.dll
 0002:000033b8       __IMPORT_DESCRIPTOR_api-ms-win-crt-stdio-l1-1-0 00000001800083b8     ucrt:api-ms-win-crt-stdio-l1-1-0.dll
 0002:000033cc       __IMPORT_DESCRIPTOR_api-ms-win-crt-string-l1-1-0 00000001800083cc     ucrt:api-ms-win-crt-string-l1-1-0.dll
 0002:000033e0       __NULL_IMPORT_DESCRIPTOR   00000001800083e0     kernel32:KERNEL32.dll
 0003:00000030       _Init_global_epoch         0000000180009030     MSVCRT:thread_safe_statics.obj
 0003:00000040       __security_cookie          0000000180009040     MSVCRT:gs_cookie.obj
 0003:00000048       __security_cookie_complement 0000000180009048     MSVCRT:gs_cookie.obj
 0003:00000050       __scrt_native_dllmain_reason 0000000180009050     MSVCRT:utility.obj
 0003:00000058       __isa_available            0000000180009058     MSVCRT:cpu_disp.obj
 0003:0000005c       __isa_enabled              000000018000905c     MSVCRT:cpu_disp.obj
 0003:00000060       __memset_fast_string_threshold 0000000180009060     MSVCRT:cpu_disp.obj
 0003:00000068       __memset_nt_threshold      0000000180009068     MSVCRT:cpu_disp.obj
 0003:00000070       __scrt_ucrt_dll_is_in_use  0000000180009070     MSVCRT:ucrt_stubs.obj
 0003:00000080       g_wrongHeapCallbacks       0000000180009080     libgcstart002.obj
 0003:00000100       g_szTagInfo                0000000180009100     libgcstart002.obj
 0003:00002040       g_tagFlags                 000000018000b040     libgcstart002.obj
 0003:00002428       g_refsToVerifyCnt          000000018000b428     libgcstart002.obj
 0003:0000242c       g_fakeUserData             000000018000b42c     libgcstart002.obj
 0003:00002430       g_tagVisitCount            000000018000b430     libgcstart002.obj
 0003:000033d0       g_refsToVerify             000000018000c3d0     libgcstart002.obj
 0003:0001aad0       g_userDataError            0000000180023ad0     libgcstart002.obj
 0003:0001aad8       mem                        0000000180023ad8     libgcstart002.obj
 0003:0001add0       ?_OptionsStorage@?1??__local_stdio_printf_options@@9@4_KA 0000000180023dd0     libgcstart002.obj
 0003:0001b398       _tls_index                 0000000180024398     MSVCRT:tlssup.obj
 0003:0001b3a0       __scrt_current_native_startup_state 00000001800243a0     MSVCRT:utility.obj
 0003:0001b3a8       __scrt_native_startup_lock 00000001800243a8     MSVCRT:utility.obj
 0003:0001b3e8       __scrt_debugger_hook_flag  00000001800243e8     MSVCRT:utility_desktop.obj
 0003:0001b3f0       ?__type_info_root_node@@3U__type_info_node@@A 00000001800243f0     MSVCRT:tncleanup.obj
 0003:0001b400       ?_OptionsStorage@?1??__local_stdio_scanf_options@@9@4_KA 0000000180024400     MSVCRT:default_local_stdio_options.obj
 0003:0001b408       __favor                    0000000180024408     MSVCRT:cpu_disp.obj
 0003:0001b410       __dyn_tls_init_callback    0000000180024410     <common>

 entry point at        0001:00003030

 Static symbols

 0000:fffd9000       .debug$S                   0000000180000000     gcstart002.exp
 0000:fffd9000       .debug$S                   0000000180000000     vcruntime:VCRUNTIME140.dll
 0000:fffd9000       .debug$S                   0000000180000000     vcruntime:VCRUNTIME140.dll
 0000:fffd9000       .debug$S                   0000000180000000     vcruntime:VCRUNTIME140.dll
 0000:fffd9000       .debug$S                   0000000180000000     vcruntime:VCRUNTIME140.dll
 0000:fffd9000       .debug$S                   0000000180000000     vcruntime:VCRUNTIME140.dll
 0000:fffd9000       .debug$S                   0000000180000000     vcruntime:VCRUNTIME140.dll
 0000:fffd9000       .debug$S                   0000000180000000     vcruntime:VCRUNTIME140.dll
 0000:fffd9000       .debug$S                   0000000180000000     ucrt:api-ms-win-crt-convert-l1-1-0.dll
 0000:fffd9000       .debug$S                   0000000180000000     ucrt:api-ms-win-crt-heap-l1-1-0.dll
 0000:fffd9000       .debug$S                   0000000180000000     ucrt:api-ms-win-crt-heap-l1-1-0.dll
 0000:fffd9000       .debug$S                   0000000180000000     ucrt:api-ms-win-crt-heap-l1-1-0.dll
 0000:fffd9000       .debug$S                   0000000180000000     ucrt:api-ms-win-crt-heap-l1-1-0.dll
 0000:fffd9000       .debug$S                   0000000180000000     ucrt:api-ms-win-crt-runtime-l1-1-0.dll
 0000:fffd9000       .debug$S                   0000000180000000     ucrt:api-ms-win-crt-runtime-l1-1-0.dll
 0000:fffd9000       .debug$S                   0000000180000000     ucrt:api-ms-win-crt-runtime-l1-1-0.dll
 0000:fffd9000       .debug$S                   0000000180000000     ucrt:api-ms-win-crt-runtime-l1-1-0.dll
 0000:fffd9000       .debug$S                   0000000180000000     ucrt:api-ms-win-crt-runtime-l1-1-0.dll
 0000:fffd9000       .debug$S                   0000000180000000     ucrt:api-ms-win-crt-runtime-l1-1-0.dll
 0000:fffd9000       .debug$S                   0000000180000000     ucrt:api-ms-win-crt-runtime-l1-1-0.dll
 0000:fffd9000       .debug$S                   0000000180000000     ucrt:api-ms-win-crt-runtime-l1-1-0.dll
 0000:fffd9000       .debug$S                   0000000180000000     ucrt:api-ms-win-crt-runtime-l1-1-0.dll
 0000:fffd9000       .debug$S                   0000000180000000     ucrt:api-ms-win-crt-runtime-l1-1-0.dll
 0000:fffd9000       .debug$S                   0000000180000000     ucrt:api-ms-win-crt-runtime-l1-1-0.dll
 0000:fffd9000       .debug$S                   0000000180000000     ucrt:api-ms-win-crt-runtime-l1-1-0.dll
 0000:fffd9000       .debug$S                   0000000180000000     ucrt:api-ms-win-crt-runtime-l1-1-0.dll
 0000:fffd9000       .debug$S                   0000000180000000     ucrt:api-ms-win-crt-runtime-l1-1-0.dll
 0000:fffd9000       .debug$S                   0000000180000000     ucrt:api-ms-win-crt-runtime-l1-1-0.dll
 0000:fffd9000       .debug$S                   0000000180000000     ucrt:api-ms-win-crt-runtime-l1-1-0.dll
 0000:fffd9000       .debug$S                   0000000180000000     ucrt:api-ms-win-crt-stdio-l1-1-0.dll
 0000:fffd9000       .debug$S                   0000000180000000     ucrt:api-ms-win-crt-stdio-l1-1-0.dll
 0000:fffd9000       .debug$S                   0000000180000000     ucrt:api-ms-win-crt-stdio-l1-1-0.dll
 0000:fffd9000       .debug$S                   0000000180000000     ucrt:api-ms-win-crt-stdio-l1-1-0.dll
 0000:fffd9000       .debug$S                   0000000180000000     ucrt:api-ms-win-crt-stdio-l1-1-0.dll
 0000:fffd9000       .debug$S                   0000000180000000     ucrt:api-ms-win-crt-stdio-l1-1-0.dll
 0000:fffd9000       .debug$S                   0000000180000000     ucrt:api-ms-win-crt-stdio-l1-1-0.dll
 0000:fffd9000       .debug$S                   0000000180000000     ucrt:api-ms-win-crt-stdio-l1-1-0.dll
 0000:fffd9000       .debug$S                   0000000180000000     ucrt:api-ms-win-crt-stdio-l1-1-0.dll
 0000:fffd9000       .debug$S                   0000000180000000     ucrt:api-ms-win-crt-stdio-l1-1-0.dll
 0000:fffd9000       .debug$S                   0000000180000000     ucrt:api-ms-win-crt-string-l1-1-0.dll
 0000:fffd9000       .debug$S                   0000000180000000     ucrt:api-ms-win-crt-string-l1-1-0.dll
 0000:fffd9000       .debug$S                   0000000180000000     ucrt:api-ms-win-crt-string-l1-1-0.dll
 0000:fffd9000       .debug$S                   0000000180000000     ucrt:api-ms-win-crt-string-l1-1-0.dll
 0000:fffd9000       .debug$S                   0000000180000000     ucrt:api-ms-win-crt-string-l1-1-0.dll
 0000:fffd9000       .debug$S                   0000000180000000     ucrt:api-ms-win-crt-string-l1-1-0.dll
 0000:fffd9000       .debug$S                   0000000180000000     ucrt:api-ms-win-crt-string-l1-1-0.dll
 0000:fffd9000       .debug$S                   0000000180000000     ucrt:api-ms-win-crt-string-l1-1-0.dll
 0000:fffd9000       .debug$S                   0000000180000000     kernel32:KERNEL32.dll
 0000:fffd9000       .debug$S                   0000000180000000     kernel32:KERNEL32.dll
 0000:fffd9000       .debug$S                   0000000180000000     kernel32:KERNEL32.dll
 0000:fffd9000       .debug$S                   0000000180000000     kernel32:KERNEL32.dll
 0000:fffd9000       .debug$S                   0000000180000000     kernel32:KERNEL32.dll
 0000:fffd9000       .debug$S                   0000000180000000     kernel32:KERNEL32.dll
 0000:fffd9000       .debug$S                   0000000180000000     kernel32:KERNEL32.dll
 0000:fffd9000       .debug$S                   0000000180000000     kernel32:KERNEL32.dll
 0000:fffd9000       .debug$S                   0000000180000000     kernel32:KERNEL32.dll
 0000:fffd9000       .debug$S                   0000000180000000     kernel32:KERNEL32.dll
 0000:fffd9000       .debug$S                   0000000180000000     kernel32:KERNEL32.dll
 0000:fffd9000       .debug$S                   0000000180000000     kernel32:KERNEL32.dll
 0000:fffd9000       .debug$S                   0000000180000000     kernel32:KERNEL32.dll
 0000:fffd9000       .debug$S                   0000000180000000     kernel32:KERNEL32.dll
 0000:fffd9000       .debug$S                   0000000180000000     kernel32:KERNEL32.dll
 0000:fffd9000       .debug$S                   0000000180000000     kernel32:KERNEL32.dll
 0000:fffd9000       .debug$S                   0000000180000000     kernel32:KERNEL32.dll
 0000:fffd9000       .debug$S                   0000000180000000     kernel32:KERNEL32.dll
 0000:fffd9000       .debug$S                   0000000180000000     kernel32:KERNEL32.dll
 0000:fffd9000       .debug$S                   0000000180000000     kernel32:KERNEL32.dll
 0000:fffd9000       .debug$S                   0000000180000000     kernel32:KERNEL32.dll
 0000:fffd9000       .debug$S                   0000000180000000     kernel32:KERNEL32.dll
 0000:fffd9000       .debug$S                   0000000180000000     kernel32:KERNEL32.dll
 0000:fffd9000       .debug$S                   0000000180000000     kernel32:KERNEL32.dll
 0000:fffd9000       .debug$S                   0000000180000000     kernel32:KERNEL32.dll
 0000:fffd9000       .debug$S                   0000000180000000     kernel32:KERNEL32.dll
 0000:fffd9000       .debug$S                   0000000180000000     kernel32:KERNEL32.dll
 0000:fffd9000       .debug$S                   0000000180000000     kernel32:KERNEL32.dll
 0001:00001210       addRefToVerify             0000000180002210 f   libgcstart002.obj
 0001:0000127c       agentThreadWrapper         000000018000227c f   libgcstart002.obj
 0001:000013e8       check_option               00000001800023e8 f   libgcstart002.obj
 0001:00001630       file_basename              0000000180002630 f   libgcstart002.obj
 0001:00002048       rawMonitorFunc             0000000180003048 f   libgcstart002.obj
 0001:00002510       startAgentThreadWrapper    0000000180003510 f   libgcstart002.obj
 0001:00002850       syncDebuggeeStatus         0000000180003850 f   libgcstart002.obj
 0001:00002af0       capture_previous_context   0000000180003af0 f   MSVCRT:gs_report.obj
 0001:00002b64       ?__scrt_initialize_thread_safe_statics@@YAHXZ 0000000180003b64 f   MSVCRT:thread_safe_statics.obj
 0001:00002c34       ?__scrt_uninitialize_thread_safe_statics@@YAXXZ 0000000180003c34 f   MSVCRT:thread_safe_statics.obj
 0001:00002ce0       $$000000                   0000000180003ce0     MSVCRT:amdsecgs.obj
 0001:00002d10       ?dllmain_crt_dispatch@@YAHQEAUHINSTANCE__@@KQEAX@Z 0000000180003d10 f   MSVCRT:dll_dllmain.obj
 0001:00002d60       ?dllmain_crt_process_attach@@YAHQEAUHINSTANCE__@@QEAX@Z 0000000180003d60 f   MSVCRT:dll_dllmain.obj
 0001:00002e78       ?dllmain_crt_process_detach@@YAH_N@Z 0000000180003e78 f   MSVCRT:dll_dllmain.obj
 0001:00002efc       ?dllmain_dispatch@@YAHQEAUHINSTANCE__@@KQEAX@Z 0000000180003efc f   MSVCRT:dll_dllmain.obj
 0001:00003910       $$000000                   0000000180004910     MSVCRT:guard_dispatch.obj
 0001:00003930       $$000000                   0000000180004930     MSVCRT:guard_xfg_dispatch.obj
 0001:00003946       ?fin$0@?0??dllmain_crt_process_attach@@YAHQEAUHINSTANCE__@@QEAX@Z@4HA 0000000180004946 f   MSVCRT:dll_dllmain.obj
 0001:0000395d       ?fin$0@?0??dllmain_crt_process_detach@@YAH_N@Z@4HA 000000018000495d f   MSVCRT:dll_dllmain.obj
 0001:00003976       ?fin$1@?0??dllmain_crt_process_detach@@YAH_N@Z@4HA 0000000180004976 f   MSVCRT:dll_dllmain.obj
 0001:0000398a       ?filt$0@?0??dllmain_dispatch@@YAHQEAUHINSTANCE__@@KQEAX@Z@4HA 000000018000498a f   MSVCRT:dll_dllmain.obj
 0001:000039c0       __scrt_is_nonwritable_in_current_image$filt$0 00000001800049c0 f   MSVCRT:utility.obj
 0002:00000218       ?__scrt_initialize_tss_var@@3P6AHXZEA 0000000180005218     MSVCRT:thread_safe_statics.obj
 0002:00000340       ?opcLengths@@3QBEB         0000000180005340     libgcstart002.obj
 0002:00002590       GS_ExceptionPointers       0000000180007590     MSVCRT:gs_report.obj
 0002:00002cc0       $unwind$fprintf            0000000180007cc0     libgcstart002.obj
 0002:00002ccc       $unwind$printf             0000000180007ccc     libgcstart002.obj
 0002:00002cd8       $unwind$?NewObject@JNIEnv_@@QEAAPEAV_jobject@@PEAV_jclass@@PEAU_jmethodID@@ZZ 0000000180007cd8     libgcstart002.obj
 0002:00002cd8       $unwind$nsk_lcomplain      0000000180007cd8     libgcstart002.obj
 0002:00002cd8       $unwind$nsk_ldisplay       0000000180007cd8     libgcstart002.obj
 0002:00002ce0       $unwind$nsk_lvdisplay      0000000180007ce0     libgcstart002.obj
 0002:00002ce0       $unwind$_RTC_Initialize    0000000180007ce0     MSVCRT:initsect.obj
 0002:00002ce0       $unwind$_RTC_Terminate     0000000180007ce0     MSVCRT:initsect.obj
 0002:00002ce0       $unwind$?__scrt_initialize_thread_safe_statics@@YAHXZ 0000000180007ce0     MSVCRT:thread_safe_statics.obj
 0002:00002cec       $unwind$nsk_complain       0000000180007cec     libgcstart002.obj
 0002:00002cec       $unwind$nsk_printf         0000000180007cec     libgcstart002.obj
 0002:00002cf4       $unwind$nsk_lvcomplain     0000000180007cf4     libgcstart002.obj
 0002:00002d0c       $unwind$nsk_ltrace         0000000180007d0c     libgcstart002.obj
 0002:00002d0c       $unwind$__report_gsfailure 0000000180007d0c     MSVCRT:gs_report.obj
 0002:00002d14       $unwind$nsk_lvtrace        0000000180007d14     libgcstart002.obj
 0002:00002d14       $unwind$__raise_securityfailure 0000000180007d14     MSVCRT:gs_report.obj
 0002:00002d14       $unwind$__scrt_initialize_crt 0000000180007d14     MSVCRT:utility.obj
 0002:00002d14       $unwind$__scrt_initialize_onexit_tables 0000000180007d14     MSVCRT:utility.obj
 0002:00002d14       $unwind$__scrt_release_startup_lock 0000000180007d14     MSVCRT:utility.obj
 0002:00002d14       $unwind$__scrt_uninitialize_crt 0000000180007d14     MSVCRT:utility.obj
 0002:00002d14       $unwind$_onexit            0000000180007d14     MSVCRT:utility.obj
 0002:00002d1c       $unwind$nsk_lverify        0000000180007d1c     libgcstart002.obj
 0002:00002d2c       $unwind$nsk_vprintf        0000000180007d2c     libgcstart002.obj
 0002:00002d3c       $unwind$?nsk_jni_lverify@@YAHHPEAUJNIEnv_@@HQEBDH1ZZ 0000000180007d3c     libgcstart002.obj
 0002:00002d50       $unwind$?nsk_jni_check_exception@@YAHPEAUJNIEnv_@@QEBDH@Z 0000000180007d50     libgcstart002.obj
 0002:00002d6c       $unwind$nsk_jvmti_parseOptions 0000000180007d6c     libgcstart002.obj
 0002:00002d88       $unwind$nsk_jvmti_createJVMTIEnv 0000000180007d88     libgcstart002.obj
 0002:00002d9c       $unwind$Java_nsk_jvmti_unit_FollowReferences_FollowRefObjects_resetTags 0000000180007d9c     libgcstart002.obj
 0002:00002d9c       $unwind$VMDeath            0000000180007d9c     libgcstart002.obj
 0002:00002d9c       $unwind$addRefToVerify     0000000180007d9c     libgcstart002.obj
 0002:00002d9c       $unwind$nsk_jvmti_resetAgentData 0000000180007d9c     libgcstart002.obj
 0002:00002d9c       $unwind$nsk_jvmti_setFailStatus 0000000180007d9c     libgcstart002.obj
 0002:00002d9c       $unwind$__scrt_initialize_default_local_stdio_options 0000000180007d9c     MSVCRT:default_local_stdio_options.obj
 0002:00002d9c       $unwind$?dllmain_crt_dispatch@@YAHQEAUHINSTANCE__@@KQEAX@Z 0000000180007d9c     MSVCRT:dll_dllmain.obj
 0002:00002d9c       $unwind$DllMain            0000000180007d9c     MSVCRT:dll_dllmain_stub.obj
 0002:00002d9c       $unwind$__GSHandlerCheck   0000000180007d9c     MSVCRT:gshandler.obj
 0002:00002d9c       $unwind$?__scrt_uninitialize_thread_safe_statics@@YAXXZ 0000000180007d9c     MSVCRT:thread_safe_statics.obj
 0002:00002d9c       $unwind$__scrt_acquire_startup_lock 0000000180007d9c     MSVCRT:utility.obj
 0002:00002d9c       $unwind$__scrt_dllmain_after_initialize_c 0000000180007d9c     MSVCRT:utility.obj
 0002:00002d9c       $unwind$__scrt_dllmain_before_initialize_c 0000000180007d9c     MSVCRT:utility.obj
 0002:00002d9c       $unwind$__scrt_dllmain_crt_thread_attach 0000000180007d9c     MSVCRT:utility.obj
 0002:00002d9c       $unwind$__scrt_dllmain_crt_thread_detach 0000000180007d9c     MSVCRT:utility.obj
 0002:00002d9c       $unwind$__scrt_dllmain_uninitialize_c 0000000180007d9c     MSVCRT:utility.obj
 0002:00002d9c       $unwind$__scrt_dllmain_uninitialize_critical 0000000180007d9c     MSVCRT:utility.obj
 0002:00002d9c       $unwind$atexit             0000000180007d9c     MSVCRT:utility.obj
 0002:00002da4       $unwind$nsk_jvmti_lverify  0000000180007da4     libgcstart002.obj
 0002:00002db8       $unwind$exitOnError        0000000180007db8     libgcstart002.obj
 0002:00002dc8       $unwind$check_option       0000000180007dc8     libgcstart002.obj
 0002:00002dc8       $unwind$_DllMainCRTStartup 0000000180007dc8     MSVCRT:dll_dllmain.obj
 0002:00002dd8       $unwind$Java_nsk_share_jvmti_ArgumentHandler_getAgentOptionsString 0000000180007dd8     libgcstart002.obj
 0002:00002dec       $unwind$Java_nsk_jvmti_unit_FollowReferences_FollowRefObjects_getTag 0000000180007dec     libgcstart002.obj
 0002:00002dec       $unwind$Java_nsk_share_jvmti_DebugeeClass_checkStatus 0000000180007dec     libgcstart002.obj
 0002:00002dec       $unwind$agentThreadWrapper 0000000180007dec     libgcstart002.obj
 0002:00002dfc       $unwind$Agent_Initialize   0000000180007dfc     libgcstart002.obj
 0002:00002dfc       $unwind$startAgentThreadWrapper 0000000180007dfc     libgcstart002.obj
 0002:00002e18       $unwind$syncDebuggeeStatus 0000000180007e18     libgcstart002.obj
 0002:00002e18       $unwind$__scrt_dllmain_exception_filter 0000000180007e18     MSVCRT:utility.obj
 0002:00002e2c       $unwind$Java_nsk_share_jvmti_DebugeeClass_resetAgentData 0000000180007e2c     libgcstart002.obj
 0002:00002e34       $unwind$MA_checkStatus     0000000180007e34     libgcstart002.obj
 0002:00002e48       $unwind$Java_nsk_jvmti_unit_FollowReferences_FollowRefObjects_setTag 0000000180007e48     libgcstart002.obj
 0002:00002e60       $unwind$Java_nsk_jvmti_unit_FollowReferences_FollowRefObjects_addRefToVerify 0000000180007e60     libgcstart002.obj
 0002:00002e7c       $unwind$rawMonitorFunc     0000000180007e7c     libgcstart002.obj
 0002:00002e94       $unwind$GarbageCollectionStart 0000000180007e94     libgcstart002.obj
 0002:00002eac       $unwind$capture_previous_context 0000000180007eac     MSVCRT:gs_report.obj
 0002:00002eb8       $unwind$__GSHandlerCheckCommon 0000000180007eb8     MSVCRT:gshandler.obj
 0002:00002ec0       $xdatasym                  0000000180007ec0     MSVCRT:amdsecgs.obj
 0002:00002ec4       $unwind$?dllmain_crt_process_attach@@YAHQEAUHINSTANCE__@@QEAX@Z 0000000180007ec4     MSVCRT:dll_dllmain.obj
 0002:00002f00       $unwind$?fin$0@?0??dllmain_crt_process_attach@@YAHQEAUHINSTANCE__@@QEAX@Z@4HA 0000000180007f00     MSVCRT:dll_dllmain.obj
 0002:00002f00       $unwind$?fin$0@?0??dllmain_crt_process_detach@@YAH_N@Z@4HA 0000000180007f00     MSVCRT:dll_dllmain.obj
 0002:00002f00       $unwind$?fin$1@?0??dllmain_crt_process_detach@@YAH_N@Z@4HA 0000000180007f00     MSVCRT:dll_dllmain.obj
 0002:00002f08       $unwind$?dllmain_crt_process_detach@@YAH_N@Z 0000000180007f08     MSVCRT:dll_dllmain.obj
 0002:00002f5c       $unwind$?dllmain_dispatch@@YAHQEAUHINSTANCE__@@KQEAX@Z 0000000180007f5c     MSVCRT:dll_dllmain.obj
 0002:00002f84       $unwind$?filt$0@?0??dllmain_dispatch@@YAHQEAUHINSTANCE__@@KQEAX@Z@4HA 0000000180007f84     MSVCRT:dll_dllmain.obj
 0002:00002f8c       $unwind$__scrt_is_nonwritable_in_current_image 0000000180007f8c     MSVCRT:utility.obj
 0002:00002fac       $unwind$__scrt_is_nonwritable_in_current_image$filt$0 0000000180007fac     MSVCRT:utility.obj
 0002:00002fb4       $unwind$__scrt_fastfail    0000000180007fb4     MSVCRT:utility_desktop.obj
 0002:00002fc4       $unwind$__security_init_cookie 0000000180007fc4     MSVCRT:gs_support.obj
 0002:00002fd0       $unwind$__isa_available_init 0000000180007fd0     MSVCRT:cpu_disp.obj
 0002:00002fe0       $xdatasym                  0000000180007fe0     MSVCRT:guard_dispatch.obj
 0002:00002fe8       $xdatasym                  0000000180007fe8     MSVCRT:guard_xfg_dispatch.obj
 0002:00002ff0       .edata                     0000000180007ff0     gcstart002.exp
 0002:00003018       rgpv                       0000000180008018     gcstart002.exp
 0002:00003050       rgszName                   0000000180008050     gcstart002.exp
 0002:00003088       rgwOrd                     0000000180008088     gcstart002.exp
 0002:000030a4       szName                     00000001800080a4     gcstart002.exp
 0002:000030b3       $N00001                    00000001800080b3     gcstart002.exp
 0002:000030c2       $N00002                    00000001800080c2     gcstart002.exp
 0002:000030cf       $N00003                    00000001800080cf     gcstart002.exp
 0002:00003114       $N00004                    0000000180008114     gcstart002.exp
 0002:00003151       $N00005                    0000000180008151     gcstart002.exp
 0002:00003199       $N00006                    0000000180008199     gcstart002.exp
 0002:000031d9       $N00007                    00000001800081d9     gcstart002.exp
 0002:00003216       $N00008                    0000000180008216     gcstart002.exp
 0002:00003251       $N00009                    0000000180008251     gcstart002.exp
 0002:0000327f       $N00010                    000000018000827f     gcstart002.exp
 0002:000032b0       $N00011                    00000001800082b0     gcstart002.exp
 0002:000032df       $N00012                    00000001800082df     gcstart002.exp
 0002:0000330e       $N00013                    000000018000830e     gcstart002.exp
 0002:00003343       $N00014                    0000000180008343     gcstart002.exp
 0002:000037aa       .idata$6                   00000001800087aa     kernel32:KERNEL32.dll
 0002:0000380e       .idata$6                   000000018000880e     vcruntime:VCRUNTIME140.dll
 0002:000039a0       .idata$6                   00000001800089a0     ucrt:api-ms-win-crt-heap-l1-1-0.dll
 0002:000039c0       .idata$6                   00000001800089c0     ucrt:api-ms-win-crt-runtime-l1-1-0.dll
 0002:000039e2       .idata$6                   00000001800089e2     ucrt:api-ms-win-crt-convert-l1-1-0.dll
 0002:00003a04       .idata$6                   0000000180008a04     ucrt:api-ms-win-crt-stdio-l1-1-0.dll
 0002:00003a24       .idata$6                   0000000180008a24     ucrt:api-ms-win-crt-string-l1-1-0.dll
 0003:00000000       ?codeAttributeName@@3PEBDEB 0000000180009000     libgcstart002.obj
 0003:00000008       ?lineNumberAttributeName@@3PEBDEB 0000000180009008     libgcstart002.obj
 0003:00000010       ?localVarAttributeName@@3PEBDEB 0000000180009010     libgcstart002.obj
 0003:00000018       ?localVarTypeAttributeName@@3PEBDEB 0000000180009018     libgcstart002.obj
 0003:00000020       ?stackMapAttributeName@@3PEBDEB 0000000180009020     libgcstart002.obj
 0003:00000028       ?callBytes@@3PAEA          0000000180009028     libgcstart002.obj
 0003:0000002c       ?allocBytes@@3PAEA         000000018000902c     libgcstart002.obj
 0003:0001aae0       nsk_context                0000000180023ae0     libgcstart002.obj
 0003:0001aaec       redefineAttempted          0000000180023aec     libgcstart002.obj
 0003:0001aaf0       redefineSucceed            0000000180023af0     libgcstart002.obj
 0003:0001aaf4       agentFailed                0000000180023af4     libgcstart002.obj
 0003:0001aaf8       agentThread                0000000180023af8     libgcstart002.obj
 0003:0001ab00       context                    0000000180023b00     libgcstart002.obj
 0003:0001abb8       agentThreadProc            0000000180023bb8     libgcstart002.obj
 0003:0001abc0       agentThreadArg             0000000180023bc0     libgcstart002.obj
 0003:0001abc8       agent_data                 0000000180023bc8     libgcstart002.obj
 0003:0001abd8       jvmti_env                  0000000180023bd8     libgcstart002.obj
 0003:0001abe0       jvm                        0000000180023be0     libgcstart002.obj
 0003:0001abe8       jni_env                    0000000180023be8     libgcstart002.obj
 0003:0001abf0       currentAgentStatus         0000000180023bf0     libgcstart002.obj
 0003:0001abf4       ?codeAttributeIndex@@3GA   0000000180023bf4     libgcstart002.obj
 0003:0001abf8       checkStatus_func           0000000180023bf8     libgcstart002.obj
 0003:0001ac00       ?lineNumberAttributeIndex@@3GA 0000000180023c00     libgcstart002.obj
 0003:0001ac04       ?localVarAttributeIndex@@3GA 0000000180023c04     libgcstart002.obj
 0003:0001ac08       ?localVarTypeAttributeIndex@@3GA 0000000180023c08     libgcstart002.obj
 0003:0001ac0c       ?stackMapAttributeIndex@@3GA 0000000180023c0c     libgcstart002.obj
 0003:0001ac10       ?stackFrameOffset@@3GA     0000000180023c10     libgcstart002.obj
 0003:0001ac14       ?mode@@3HA                 0000000180023c14     libgcstart002.obj
 0003:0001ac18       ?orig@@3PEBEEB             0000000180023c18     libgcstart002.obj
 0003:0001ac20       ?gen@@3PEAEEA              0000000180023c20     libgcstart002.obj
 0003:0001ac28       ?inputPos@@3PEAEEA         0000000180023c28     libgcstart002.obj
 0003:0001ac30       ?endPos@@3PEBEEB           0000000180023c30     libgcstart002.obj
 0003:0001ac38       ?genPos@@3PEAEEA           0000000180023c38     libgcstart002.obj
 0003:0001ac40       ?markPos@@3PEAEEA          0000000180023c40     libgcstart002.obj
 0003:0001ac48       ?constantPool@@3PEAPEADEA  0000000180023c48     libgcstart002.obj
 0003:0001ac50       ?constantPoolSize@@3GA     0000000180023c50     libgcstart002.obj
 0003:0001ac54       ?constantPoolCount@@3GA    0000000180023c54     libgcstart002.obj
 0003:0001ac58       ?zeroBytes@@3PAEA          0000000180023c58     libgcstart002.obj
 0003:0001ac5c       ?codeLength@@3IA           0000000180023c5c     libgcstart002.obj
 0003:0001ac60       ?map@@3PEAIEA              0000000180023c60     libgcstart002.obj
 0003:0001ac68       ?widening@@3PEACEA         0000000180023c68     libgcstart002.obj
 0003:0001ac70       jvmti                      0000000180023c70     libgcstart002.obj
 0003:0001ac78       result                     0000000180023c78     libgcstart002.obj
 0003:0001ac80       callbacks                  0000000180023c80     libgcstart002.obj
 0003:0001adb8       caps                       0000000180023db8     libgcstart002.obj
 0003:0001adc8       gcstart                    0000000180023dc8     libgcstart002.obj
 0003:0001ade0       GS_ExceptionRecord         0000000180023de0     MSVCRT:gs_report.obj
 0003:0001ae80       GS_ContextRecord           0000000180023e80     MSVCRT:gs_report.obj
 0003:0001b350       ?g_tss_cv@@3U_RTL_CONDITION_VARIABLE@@A 0000000180024350     MSVCRT:thread_safe_statics.obj
 0003:0001b358       ?g_tss_event@@3PEAXEA      0000000180024358     MSVCRT:thread_safe_statics.obj
 0003:0001b360       ?g_tss_mutex@@3U_RTL_CRITICAL_SECTION@@A 0000000180024360     MSVCRT:thread_safe_statics.obj
 0003:0001b388       ?g_sleep_condition_variable_cs@@3P6AHPEAU_RTL_CONDITION_VARIABLE@@PEAU_RTL_CRITICAL_SECTION@@K@ZEA 0000000180024388     MSVCRT:thread_safe_statics.obj
 0003:0001b390       ?g_wake_all_condition_variable@@3P6AXPEAU_RTL_CONDITION_VARIABLE@@@ZEA 0000000180024390     MSVCRT:thread_safe_statics.obj
 0003:0001b39c       ?__proc_attached@@3HA      000000018002439c     MSVCRT:dll_dllmain.obj
 0003:0001b3b0       ?is_initialized_as_dll@@3_NA 00000001800243b0     MSVCRT:utility.obj
 0003:0001b3b1       ?module_local_atexit_table_initialized@@3_NA 00000001800243b1     MSVCRT:utility.obj
 0003:0001b3b8       ?module_local_atexit_table@@3U_onexit_table_t@@A 00000001800243b8     MSVCRT:utility.obj
 0003:0001b3d0       ?module_local_at_quick_exit_table@@3U_onexit_table_t@@A 00000001800243d0     MSVCRT:utility.obj
